:100000002CC044C043C042C041C040C03FC03EC0FD
:100010003DC03CC03BC03AC039C038C037C036C014
:1000200035C034C033C057524F4E470A004F4B21A2
:100030000A005472792025690A0052656164792E9C
:100040000A0045464765666700202B2D2E30313269
:100050003334353637383968000011241FBECFEDF0
:10006000CDBF10E0A0E6B0E0E0EBF5E002C0059007
:100070000D92AE36B107D9F710E0AEE6B0E001C0A0
:100080001D92A437B107E1F706D090C2B9CF5F9BAC
:10009000FECF8CB10895AF92BF92CF92DF92EF92D4
:1000A000FF920F931F93CF93DF9383E390E06CD085
:1000B00000D08AE390E0EDB7FEB792838183F3D15D
:1000C000C0E0D0E00F900F9022E3A22E20E0B22EED
:1000D00008EC10E09DE2C92E90E0D92E86E2E82ED1
:1000E00080E0F82E00D000D0EDB7FEB7B282A1823A
:1000F000D483C383D8D10F900F900F900F905F9B44
:10010000FECF8CB18133E1F45F9BFECF8CB18433A1
:10011000B9F45F9BFECF8CB1873391F45F9BFECF28
:100120008CB1813369F480E29EE4F8013197F1F7F4
:100130000197D9F700D0EDB7FEB7D282C1820CC0CB
:1001400080E29EE4F8013197F1F70197D9F700D0EA
:10015000EDB7FEB7F282E182A6D10F900F9003C0F7
:100160005F9BFECF8CB15F99FBCF2196BBCF1F93D6
:10017000182F8A3011F48DE0FADF5D9BFECF1CB999
:1001800080E090E01F91089528E12AB989B9892F6C
:10019000990F990B82B980E690E09093710080935B
:1001A00070000895ABE0B0E0E7EDF0E012C15C0153
:1001B0004B017A01FC0117821682838181FD08C000
:1001C0006FEF7FEFFEC042E050E0E40EF51E04C08A
:1001D0003E010894611C711CF501D380F401D3FC2D
:1001E0008591D3FE81914F01882309F4E7C08532C0
:1001F00059F4D3FC6591D3FE61914F01653219F03A
:10020000062F10E01AC085E290E029C0002309F40F
:10021000D5C089E490E0602F70E00ED1892B39F4CD
:10022000033211F4106103C00C3661F41068F4015C
:10023000D3FC0591D3FE01914F0117FFE7CF0023B7
:1002400009F4BCC082E490E0602F70E0F5D0892B07
:1002500049F044E050E0E40EF51E8FE390E0B50174
:10026000F6D0BACF033629F0033771F00335E1F445
:100270000AC087010E5F1F4FF70180819181B50190
:10028000E6D07801A9CF1160F701C080D18003C00A
:1002900090E0B501DCD0F60110FD859110FF819151
:1002A0006F018823A9F78FCF043611F0093639F58D
:1002B00017FF08C0F701208131814281538184E01A
:1002C00090E00AC0F701808191819C01442737FDAD
:1002D0004095542F82E090E0E80EF91E1F7E57FFF4
:1002E00008C050954095309521953F4F4F4F5F4F37
:1002F0001064CA01B901A3012AE030E034C000371C
:10030000A9F0013730F40835B1F00F3609F056C0C6
:1003100006C0053739F0083709F050C008C028E09A
:1003200030E00CC01F7E2AE030E008C0106114628B
:1003300020E130E003C0146020E132E017FF08C084
:10034000F701608171818281938144E050E008C0AF
:10035000F70180819181BC0180E090E042E050E0B3
:10036000E40EF51EA301C2D0D82ED618012F10E03E
:1003700006FF04C08DE290E0B50169D004FF13C010
:10038000FE01ED0DF11D8081803369F080E390E086
:10039000B5015DD002FF07C000721070C801885A15
:1003A0009F4FB50154D0DA94F301ED0DF11D80811A
:1003B00090E0B5014CD0DD20B1F70ECFF50166819C
:1003C0007781CB012B96EEE020C02F923F924F9287
:1003D0005F926F927F928F929F92AF92BF92CF92D5
:1003E000DF92EF92FF920F931F93CF93DF93CDB7DE
:1003F000DEB7CA1BDB0B0FB6F894DEBF0FBECDBF56
:1004000009942A88398848885F846E847D848C8426
:100410009B84AA84B984C884DF80EE80FD800C812F
:100420001B81AA81B981CE0FD11D0FB6F894DEBF12
:100430000FBECDBFED010895FC010590061621F019
:100440000020D9F7C00108953197CF0108950F9387
:100450001F93CF93DF938C01EB018B8181FF1BC036
:1004600082FF0DC02E813F818C819D812817390725
:1004700064F4E881F9810193F983E88306C0E88593
:10048000F985802F0995892B31F48E819F81019602
:100490009F838E8302C00FEF1FEFC801DF91CF91C2
:1004A0001F910F910895A0E0B0E0E8E5F2E09DCF44
:1004B000FE01359661917191A0917000B09171002B
:1004C00013968C911397886013968C93809170008B
:1004D00090917100AF0166DEE0917000F0917100C3
:1004E0002381277F23832096E2E09BCFFA01AA276E
:1004F000283061F1203191F1E8946F936E7F6E5F47
:100500007F4F8F4F9F4FAF4FB1E040D0B4E03ED010
:10051000670F781F891F9A1FA11D680F791F8A1FF7
:10052000911DA11D6A0F711D811D911DA11D22D05C
:1005300009F468943F91062E000C3019000C000C51
:100540003019305D3193CEF6CF010895462F4770B4
:10055000405D4193B3E00FD0C9F7F6CF462F4F70FF
:10056000405D4A3318F0495D31FD4052419302D05D
:10057000A9F7EACFB4E0A695979587957795679503
:10058000BA95C9F700976105710508959B01AC0103
:100590000A2E06945795479537952795BA95C9F72A
:1005A000620F731F841F951FA01D0895F894FFCF3D
:0E05B0000000000200000000B7000000000084
:00000001FF
